:100000001AC033C032C07CC230C02FC0C3C12DC0A3
:100010002CC02BC02AC074C59DC527C026C025C0D2
:1000200024C023C022C00A0020002000200020207D
:1000300000200020000011241FBECFE5D4E0DEBF69
:10004000CDBF10E0A0E6B0E0EAEFFCE002C0059012
:100050000D92A436B107D9F711E0A4E6B0E001C0D3
:100060001D92A737B107E1F7D1C4CACFBC011092E6
:10007000E3001092E200482F8093240110C0369ACA
:100080003699FECF8091E2009091E30024B135B122
:10009000820F931F9093E3008093E200415044232A
:1000A00071F7109224018091E2009091E30011D643
:1000B0007093E3006093E2008091E2009091E3008E
:1000C000089510922401FC016150704009C08281A2
:1000D000938181939193809124018F5F8093240178
:1000E0008091240199278617970788F38091E20071
:1000F0009091E300918380830895FC011092E300C6
:100100001092E200109224010FC08091E2009091C1
:10011000E30021913191820F931F9093E30080932C
:10012000E2004F5F4093240140912401842F9927DE
:100130008617970750F38091E2009091E300C9D5AC
:100140007093E3006093E2008091E2009091E300FD
:10015000089582E88FBD89E08EBD84E090E09BBD6C
:100160008ABD85B5886085BD85B5876085BD8CE90C
:1001700083BD89B7806889BF88B7806888BF0895C4
:1001800084E08EBD8AE78BBD82E18ABD8EB5886032
:100190008EBD89B7806189BF88B7806188BF18BA72
:1001A00008952091750130917601E091E6009091DB
:1001B00049013FC02F5F3F4F82990CC0809166007C
:1001C00080FD08C09F5F809166008160809366001B
:1001D00020E030E0992311F484E203C0913019F457
:1001E00088E288BB07C0923011F480E3FACF9330E5
:1001F00009F490E0829B0DC08AEF2030380759F453
:100200008091660080FF05C0809166008E7F80939C
:10021000660020E030E083990CC0E92FFF27E05A08
:10022000FF4FE0818091660082608093660020E04D
:1002300030E08091660081FFBDCF3093760120933E
:100240007501E093E600909349010895949A82E045
:1002500087B91092EE001092ED0088E28093E400DE
:100260008EE190E003DF8091ED009091EE0020910F
:10027000E2003091E300820F931F9093EE00809391
:10028000ED008091E40081508093E400882341F7E1
:100290008091ED009091EE0068E270E01AD57093C5
:1002A000F0006093EF0094988091EF009091F0003F
:1002B000C99758F4809166008064809366008091AD
:1002C00067008460809367005BDF8091EF0090910E
:1002D000F0008638910558F0809166008064809324
:1002E00066008091670088608093670049DF809195
:1002F000660086FD4EC081E087B91092EE00109234
:10030000ED0088E28093E4008EE190E0AFDE809122
:10031000ED009091EE002091E2003091E300820F19
:10032000931F9093EE008093ED008091E400815044
:100330008093E400882341F78091ED009091EE00D6
:1003400068E270E0C6D4709323016093220180912B
:1003500022019091230189549340A8F480912201B5
:1003600090912301873E910560F480916600806141
:10037000809366008091660080648093660000DF51
:100380000895E7DE08958091660080688093660096
:10039000F7DE08951F920F920FB60F9211242F933C
:1003A0003F934F935F936F937F938F939F93AF93FD
:1003B000BF93EF93FF938091660086FF20C08091EA
:1003C000670082FF04C088B390E3892788BB8091CF
:1003D000670083FF04C088B398E3892788BB8091B6
:1003E000660084FF04C088B39CE3892788BB8091A2
:1003F000670080FF04C088B39CE2892788BB809196
:10040000660087FF6CC060917501709176016F5F27
:100410007F4F709376016093750148B32091490135
:1004200033272E5F3F4F81E090E002C0880F991F75
:100430002A95E2F78062482748BB6430710511F4C1
:10044000949808C06530710528F0949A109276014E
:1004500010927501949943C081E087B98CE390E0D4
:1004600005DE8091E2009091E30090932301809358
:10047000220182E087B980EF90E0F8DD8091E20010
:100480009091E3009093F0008093EF0080916600DC
:1004900084608093660080912201909123018954A9
:1004A0009340E8F4809166008062809366001EBCF1
:1004B00089B78F7E89BF88B78F7E88BF48B3209168
:1004C000490133272E5F3F4F81E090E002C0880F43
:1004D000991F2A95E2F7482B48BB39983ADEFF91DD
:1004E000EF91BF91AF919F918F917F916F915F91AC
:1004F0004F913F912F910F900FBE0F901F90189525
:100500001F920F920FB60F9211242F933F934F9388
:100510005F936F937F938F939F93AF93BF93EF936B
:10052000FF9320917501309176012F5F3F4F3093FB
:100530007601209375018091660083FD43C02430CD
:10054000310508F43FC017B88AE590E08FDD80914F
:10055000E2009091E3009093260180932501209181
:100560002501309126018091AD009091AE00029658
:100570008217930768F48AB59BB501979BBD8ABD26
:100580008AB59BB5039720F483E090E09BBD8ABDBC
:1005900020912501309126018091AD009091AE000F
:1005A00003972817390770F48AB59BB501969BBD50
:1005B0008ABD8AB59BB5895E934020F088EE93E0B2
:1005C0009BBD8ABD4091750150917601453551051D
:1005D00079F4809125019091260190934E018093AA
:1005E0004D018AB59BB5909365008093640034C03B
:1005F0004735510561F580911F018F5F80931F0181
:1006000080911F01893059F48091AD009091AE0026
:1006100001969093AE008093AD0010921F0120913F
:10062000AD003091AE008091E60099272817390778
:1006300020F09093AE008093AD00809166008860BA
:10064000809366001BBC1ABC1FBC1EBC0AC0493587
:10065000510511F4979AB6C14A35510511F497988E
:10066000B1C14B355105B9F482E087B986E490E019
:10067000FDDC69E170E080EB90E023DD69E170E092
:1006800080EB90E03ADD8091E2009091E30090935E
:10069000F0008093EF0080917501909176018C3588
:1006A0009105F9F481E087B988E290E0DFDC65E14B
:1006B00070E081EF90E005DD65E170E081EF90E0B2
:1006C0001CDD8091E2009091E300909328018093DB
:1006D0002701809127019091280190932301809315
:1006E000220180917501909176018D35910509F077
:1006F0004BC183E087B98DE290E0B8DC60E170E047
:1007000089E291E0DEDC60E170E089E291E0F5DC15
:100710008091E2009091E3009093660180936501DF
:1007200080912201909123018E5D934068F1809128
:100730006700816080936700809166008064809389
:100740006600109265001092640085B5877F85BDB4
:1007500085B585BD89B78F7789BF88B78F7788BF03
:1007600048B32091490133272E5F3F4F81E090E04D
:1007700002C0880F991F2A95E2F780958F6D482354
:1007800048BB1FBC1EBCB9988091EF009091F0004F
:100790008239910568F180916700886080936700D5
:1007A00080916600806480936600109265001092CC
:1007B000640085B5877F85BD85B585BD89B78F7791
:1007C00089BF88B78F7788BF48B320914901332705
:1007D0002E5F3F4F81E090E002C0880F991F2A955D
:1007E000E2F780958F6D482348BB1FBC1EBCB998AB
:1007F0008091EC008F3070F080916D0190916E01CE
:100800002091650130916601820F931F90936E01D4
:1008100080936D018091EC008F5F8093EC0080915C
:10082000EC00893109F0ABC08091710190917201A7
:100830009093700180936F0180916D0190916E0192
:100840006AE070E046D270936E0160936D01809112
:100850006D0190916E01909372018093710180916E
:1008600071019091720120916F0130917001821B92
:10087000930B2AE030E0AC01429FC001439F900DF2
:10088000529F900D11249093740180937301809175
:1008900073019091740197FD0EC080917301909146
:1008A0007401815991403CF480912201909123017F
:1008B000815B934020F41092740110927301809137
:1008C000690190916A01909368018093670180911A
:1008D0006B0190916C0190936A0180936901809102
:1008E00073019091740190936C0180936B018091DE
:1008F0006701909168012091690130916A014091EE
:100900006B0150916C01820F931F840F951F63E060
:1009100070E0DFD1709374016093730110926E01E7
:1009200010926D011092EC0080914A018F5F8093CC
:100930004A0120917301309174018091AF00992791
:100940002817390714F010924A0180917301909191
:1009500074018093AF0080914A01833081F485B5A2
:10096000877F85BD85B585BD89B78F7789BF88B7F6
:100970008F7788BF1FBC1EBC88B38C6388BB8091F7
:100980006600846080936600809175019091760185
:1009900084369105B9F482E88FBD89E08EBD8091DF
:1009A0006600877F80936600809164009091650067
:1009B0009BBD8ABD88B390E2892788BB10927601DF
:1009C00010927501FF91EF91BF91AF919F918F911F
:1009D0007F916F915F914F913F912F910F900FBE3B
:1009E0000F901F90189514BA15BA8FEF87BB80E24D
:1009F00088BB80EF81BB8FE682BB309A319A329AF6
:100A0000379A87E690E0CBD078940895CFE5D4E08C
:100A1000DEBFCDBFE8DFC5DB19DC8091660082FF59
:100A2000FCCF80914D0190914E014AE050E067EE7D
:100A300070E02BD187EE90E0F0D083E390E0F9D026
:100A400080916400909165004AE050E067EE70E0AC
:100A50001CD187EE90E0E1D081E390E0EAD0809174
:100A60002201909123014AE050E067EE70E00DD141
:100A700087EE90E0D2D08EE290E0DBD080917101E1
:100A8000909172014AE050E067EE70E0FED087EE90
:100A900090E0C3D08CE290E0CCD080917301909133
:100AA00074014AE050E067EE70E0D0D087EE90E04D
:100AB000B4D08AE290E0BDD080916501909166014A
:100AC0004AE050E067EE70E0E0D087EE90E0A5D01D
:100AD00088E290E0AED08091EF009091F0004AE083
:100AE00050E067EE70E0D1D087EE90E096D086E2DD
:100AF00090E09FD0809166008B7F809366008DCFC1
:100B00001F920F920FB60F9211242F938F939F93E2
:100B1000EF93FF939BB12CB1E091AA00EF5FEF71CF
:100B20008091AB00E81711F482E008C0892F88712A
:100B3000E093AA00FF27E857FF4F20838093AC0083
:100B4000FF91EF919F918F912F910F900FBE0F907A
:100B50001F9018951F920F920FB60F9211248F932A
:100B60009F93EF93FF939091A8008091A90098170D
:100B700061F0E091A900EF5FEF71E093A900FF271A
:100B8000E859FF4F80818CB901C05598FF91EF91D2
:100B90009F918F910F900FBE0F901F9018951092FC
:100BA000A8001092A9001092AA001092AB00292F61
:100BB000332720BD89B988E98AB986E880BD0895C0
:100BC0009091AA008091AB00981719F480E091E011
:100BD0000895E091AB00EF5FEF71E093AB00FF276A
:100BE000E857FF4F20818091AC009927982F8827E4
:100BF000820F911D0895282F9091A8009F5F9F71EB
:100C00008091A9009817E1F3E92FFF27E859FF4FDA
:100C100020839093A800559A0895CF93DF93EC0119
:100C200002C02196E8DF88818823D9F7DF91CF9130
:100C30000895CF93DF93EC0101C0DDDFFE01219623
:100C400084918823D1F7DF91CF910895FB019F0113
:100C5000E8944230BCF04532ACF44A3029F497FBBA
:100C60001EF4909581959F4F642F772732D0805D39
:100C70008A330CF0895D8193CB010097A9F716F4B4
:100C80005DE251931082C90114C0FB019F01423003
:100C90006CF045325CF4642F77271BD0805D8A337B
:100CA0000CF0895D8193CB010097A9F71082C901EF
:100CB00000C0DC01FC0101900020E9F73297AE177B
:100CC000BF0730F47C916081708331976D93F7CFCB
:100CD0000895AA1BBB1B51E107C0AA1FBB1FA61783
:100CE000B70710F0A61BB70B881F991F5A95A9F7D5
:0A0CF00080959095BC01CD01089598
:040CFA002D46500033
:00000001FF
